:100000008031E82A0000203085000A308400000892
:10001000031918280330F800F701F70B0D28F80B27
:100020000C283C30F700F70B13281628800B0A2801
:100030000800970196010A30AA0003201708FA0069
:100040001608F70017087A02031D1E287708A70074
:100050007A08A800A9012808003C03184328FF3AA1
:10006000031D36282708383C031843282808013C7C
:10007000031C4328031D40282708463C031C432833
:100080000130A90032292808003C03185B28FF3AF8
:10009000031D4E282708AF3C03185B282808013CA5
:1000A000031C5B28031D58282708C13C031C5B2840
:1000B0000230A90032292808003C03187328FF3AAF
:1000C000031D66282708D53C031873282808013C1F
:1000D000031C7328031D70282708E93C031C7328A0
:1000E0000330A90032292808023C03188B28FF3A64
:1000F000031D7E2827085F3C03188B282808033C33
:10010000031C8B28031D88282708833C031C8B288D
:100110000430A90032292808023C0318A328FF3A1A
:10012000031D96282708AB3C0318A3282808033C86
:10013000031CA328031DA0282708D33C031CA328C5
:100140000530A90032292808053C0318BB28FF3ACE
:10015000031DAE282708BF3C0318BB282808073C0E
:10016000031CBB28031DB8282708073C031CBB2819
:100170000630A90032292808063C0318D328FF3A84
:10018000031DC6282708583C0318D3282808073C15
:10019000031CD328031DD0282708A63C031CD32802
:1001A0000730A900322928080C3C0318EB28FF3A35
:1001B000031DDE282708803C0318EB2828080E3C86
:1001C000031CEB28031DE82827080E3C031CEB2822
:1001D0000830A900322928080D3C03180329FF3AEA
:1001E000031DF6282708B23C0318032928080F3CF2
:1001F000031C0329031D002927084C3C031C032969
:100200000930A900322928081A3C03181B29FF3A93
:10021000031D0E292708013C03181B2928081C3C34
:10022000031C1B29031D182927081D3C031C1B291F
:100230000A30A900322928081C3C03183229FF3A49
:10024000031D26292708653C0318322928081E3C6F
:10025000031C3229031D30292708993C031C32292D
:100260000B30A9002908F8000800A71D3B2922002F
:100270000C153D29200022000C112000271D4429C7
:1002800022000C154629200022008C112000A71CFA
:100290004D2922008C154F29200022000C1220002D
:1002A000271C562922000D165829200022000D1265
:1002B00020000800A9080319BA292908033A0319DC
:1002C0007729073A03197D290C3A031986290E3A32
:1002D00003198D290C3A031991290B3A031998290E
:1002E000113A0319A129123A0319A729B1292200A9
:1002F0008C1021008C100C14BA2922008C102100C3
:100300008C1022000C1421000C10BA2921008C142E
:1003100022000C1021000C10BA2921008C140C149E
:10032000BA2921008C1422000C1421000C10BA29C7
:1003300022008C1421008C1022000C1021000C10C3
:10034000BA2922008C1421008C100C14BA29220026
:100350008C1421008C1022000C1421000C10BA29DE
:10036000200022008C1021008C1022000C10210093
:100370000C10BA29200008002708003A0319D629D2
:10038000013A0319DA29033A0319DE29013A03195C
:10039000E229073A0319E629013A0319EA29033A3F
:1003A0000319EE29013A0319F229F6290130A900AF
:1003B0005A21F7290230A9005A21F7290330A90050
:1003C0005A21F7290430A9005A21F7290630A9003B
:1003D0005A21F7290830A9005A21F7290A30A90023
:1003E0005A21F7291030A9005A21F729F72980311D
:1003F000302B2808013A03191C2A033A03193C2A16
:10040000013A03193C2A073A03195C2A013A0319F5
:100410005C2A033A03197C2A013A03197C2A0F3A11
:1004200003199C2A013A03199C2A033A0319BC2A8E
:10043000013A0319BC2ADC2A2708033903192A2A9E
:10044000013A03192E2A033A0319322A013A0319F1
:10045000362A3A2A1030A9005A213B2A1030A90026
:100460005A213B2A1030A9005A213B2A1030A900FA
:100470005A213B2A3B2AE62A2708033903194A2A2C
:10048000013A03194E2A033A0319522A013A031971
:10049000562A5A2A0430A9005A215B2A1030A90092
:1004A0005A215B2A0830A9005A215B2A0830A9008A
:1004B0005A215B2A5B2AE62A2708033903196A2A8C
:1004C000013A03196E2A033A0319722A013A0319F1
:1004D000762A7A2A0430A9005A217B2A0830A900FA
:1004E0005A217B2A0830A9005A217B2A0430A9000E
:1004F0005A217B2A7B2AE62A2708033903198A2AEC
:10050000013A03198E2A033A0319922A013A031970
:10051000962A9A2A0430A9005A219B2A0430A9005D
:100520005A219B2A0430A9005A219B2A0230A90093
:100530005A219B2A9B2AE62A270803390319AA2A4B
:10054000013A0319AE2A033A0319B22A013A0319F0
:10055000B62ABA2A0230A9005A21BB2A0230A900C1
:100560005A21BB2A0230A9005A21BB2A0130A90016
:100570005A21BB2ABB2AE62A270803390319CA2AAB
:10058000013A0319CE2A033A0319D22A013A031970
:10059000D62ADA2A0130A9005A21DB2A0130A90023
:1005A0005A21DB2A0130A9005A21DB2A0130A90097
:1005B0005A21DB2ADB2AE62A271DE22A0430A90079
:1005C0005A21E52A0230A9005A21E62A80314C2B13
:1005D000850184011F30830523008C018D012200D9
:1005E00092019101940193010A302000A400A5001A
:1005F0001430A6002100990164302000AA000320D5
:10060000FF3021008C008D0024008D002100951307
:10061000853020009800990121000C118C110C12DA
:100620000D122000A2010D1C22158D1CA2140D1DFF
:100630002214A3018D19A30AA308031D352B192029
:100640007808A1002108A700352122082402031DF3
:100650002D2B250823020319302B2208A700BC29C3
:100660002208A4002308A500522B19207808A10015
:100670002108A700352121082602031D472B220847
:100680002402031D472B250823020319522B22089D
:10069000A7002108A800F9292108A6002208A40023
:0806A0002308A500122B6300E2
:020000040001F9
:04000E000239FF1E96
:00000001FF
